:1000000008C3000024C300000C941E0920C3000094
:100010001EC300001CC300001AC3000018C3000068
:1000200016C3000014C300000C948E0D0C94BC0E7B
:100030000EC300000CC300000AC3000008C3000088
:1000400006C300000C94620902C3000000C3000054
:10005000FEC200000C94DB0AFAC20000F8C20000E5
:10006000F6C20000F4C20000F2C20000F0C20000BC
:10007000EEC20000ECC200000C94D614E8C20000EE
:10008000C3C50000E4C20000E2C20000E0C20000FC
:10009000DEC20000DCC2000000291E1F2021222336
:1000A000242526272D2E2A2B141A0815171C180C68
:1000B00012132F3028E0041607090A0B0D0E0F3318
:1000C0003435E1311D1B0619051110363738E55559
:1000D000E22C393A3B3C3D3E3F4041424353475F6F
:1000E0006061565C5D5E57595A5B6263C2BE644490
:1000F0004567B0B28CB7B8B9BABBBCBD68696A6BAA
:100100006C6D6E6F707172C188B1B387B4B5739343
:10011000928ABF8BB68985C00142003E3C3A3B457E
:100120006843413F3D2B356769E2E188E0141EB02A
:100130006AB11D16041A1FB26B061B070821208C1A
:100140006C2C1909171522B76D11050B0A1C23B861
:100150006EB3100D182425B96F360E0C122726BA6F
:100160007037380F33132DBB718734B42F2EBC7208
:1001700039E52830B531BD73BE6493928ABF2A8BAE
:10018000B659895C5F85C0C162635A5D5E60295360
:1001900044575B565561470000000040C200000014
:1001A00000000000000000000000000000F9E60070
:1001B00000E4E90000FF000000000000E3FEF000A2
:1001C000EC000000E7FD0000F700000065FC00EF18
:1001D00000EB000066FB00FAEA000000A9F800004E
:1001E0000000000000F600540000E80000F50000E8
:1001F0000000000000000058000000AA00000000FD
:100200000000000000004D00504A000000494C5121
:10021000004F52000000004E00464B4801BF00BB9B
:10022000B9B7B83A68C0BEBCBA2B353B69E0E164E7
:1002300039141E3C6AE21D16041A1F3D6B061B078B
:100240000821203E6C2C19091715223F6D11050B52
:100250000A1C23406EE6100D182425416F360E0C43
:10026000122726427037380F33132D4371873432EB
:100270002F2E4472E4E52830318945735150935252
:100280004C4D2A49B6594F5C5F4E4A4B62635A5DEA
:100290005E602953B2575B5655614700000000BDB0
:1002A000C20A4D6F64653A2041542F5053320A0AF6
:1002B000000A4D6F64653A2050432F58540A0A00D3
:1002C000756E6B6E6F776E00322028657874656E80
:1002D0006465642900436F6465205365743A2000A7
:1002E0004B6579626F6172642049443A20000001D5
:1002F0000000580312000200006A0374002200008C
:10030000DE0312002100007C030900220100F0033B
:100310001500210100950309002202000504DC00FC
:10032000210200AE030900220300E1041C002103A6
:1003300000C7030900030000FD04040103090401D0
:10034000050E0203090411053801C10601C1260189
:10035000C12601C13601C036120100020000002092
:10036000C0167D04000101020001090274000401AD
:1003700000A032090400000103010100092111015C
:100380000001221200070581030800010904010091
:1003900001030000000921110100012215000705D9
:1003A0008303200001090402000103000000092169
:1003B0001101000122DC0007058203170001090476
:1003C00003000203000000092111010001221C00AA
:1003D00007058403400002070505034000080501E6
:1003E0000906A101150026FF00950875088103C0C4
:1003F0000631FF0974A1537508150026FF009520EA
:1004000009758102C005010906A1018501750195E3
:1004100008050719E029E7150025018102950575F2
:1004200001050819012905910295017503910375CC
:100430000195310507190129311500250181029522
:1004400001750181037501956905071933299B150C
:10045000002501810295017501810375019508054B
:1004600007199D29A41500250181029504750181B4
:1004700003C005010980A101850275019503198159
:100480002983150025018102950575018103C005A9
:100490000C0901A10185037501951809B509B60973
:1004A000B709CD09E209E509E709E909EA0A5201B4
:1004B0000A53010A54010A55010A83010A8A010AF2
:1004C00092010A94010A21020A23020A24020A253F
:1004D000020A26020A27020A2A02150025018102C1
:1004E000C00699FF0A6824A1017508150026FF00BF
:1004F000954009018102954009029102C004030957
:10050000040E0353006F006100720065007200006A
:1005100000380353006F006100720065007200270D
:1005200000730020004B006500790062006F0061DD
:100530000072006400200043006F006E00760065CA
:100540000072007400650072000000616C6C6F63E3
:10055000206F6B2E0A00616C6C6F63206661696CA2
:1005600065642E0A00616C6C6F63206661696C655E
:10057000642E0A00746F74616C5F6D6163726F73D7
:100580003A20006D61785F6C617965723A20006C89
:1005900061796572646566733A2000216170706CE0
:1005A000790A006C656E3C350A000A0A72656D6155
:1005B000696E696E673A20006572726F722000651D
:1005C00072726F7220006572726F7220002169640E
:1005D00020002173657420002173656C65637420AD
:1005E000006D6163726F73200072656D61707320BE
:1005F000006C6179657273200003010001010C0237
:10060000010104000005002007000006001008009A
:10061000000011241FBECFEFD0E2DEBFCDBF11E03E
:10062000A0E0B1E0E8E8F8E300E00BBF02C007900B
:100630000D92A032B107D9F713E0A0E2B1E001C0FA
:100640001D92AB3AB107E1F7AAD00C94421CD8CC6A
:1006500090910001923021F1933018F4913041F5DE
:1006600005C0933059F0943019F510C087FD20C0B3
:10067000E82FF0E0E856FF4F849108958538C0F4E4
:10068000E82FF0E0E45EFD4F84910895662341F089
:100690008F3770F4E82FF0E0E356FE4F8491089511
:1006A000853830F4E82FF0E0E85EFE4F849108953D
:1006B00080E008950E94451A0E944F1A109222016C
:1006C000109223011092240108951F93182F0E9465
:1006D0003E1A212F30E0882371F08AB188638AB9ED
:1006E0009BB143E0220F331F4A95E1F7822F8873B5
:1006F000977C892B0DC09AB183E0220F331F8A9516
:10070000E1F7822F8873977C892B8AB98BB1886334
:100710008BB91F9108959CDF0C94521A99DF0C94A9
:10072000711ACF92DF92EF92FF920F931F93CF93A4
:10073000DF93ABD2082F80912601802739F1C0E0EA
:10074000D0E01BEAC82EDD24E02EFF24C6010C2ECB
:1007500002C0959587950A94E2F780FF10C0C70103
:100760000C2E02C0959587950A94E2F780FF04C08D
:10077000812F0E94521A03C0812F0E94711A219664
:100780001F5F103B19F70093260181E0DF91CF91A5
:100790001F910F91FF90EF90DF90CF9008952F92CF
:1007A0003F924F925F926F927F928F929F92AF9201
:1007B000BF92CF92DF92EF92FF920F931F93DF933E
:1007C000CF9300D00F92CDB7DEB780E88093610061
:1007D00010926100569A80E078DF87E076DFDDD600
:1007E0000E94411A5AD536D265DF80E076D2332492
:1007F000882499245524AA24BB24650114E0412EA1
:10080000B2E02B2E3320A1F42FB7F894809136015B
:1008100090913701A0913801B09139012FBF855FC8
:100820009140A040B04020F081E057D2332433946F
:10083000882009F0E5C02FB7F89480913601909197
:100840003701A0913801B09139012FBF895B9B40DE
:10085000A040B04008F4D4C00E94EC15982F9F70BF
:1008600099F082958F7059F490930001913019F4AA
:100870002092290161C081E0809329015DC08093AD
:1008800029019093000158C010920001109221019B
:10089000109220018EEE62E355D5823009F041C0FE
:1008A00082E3FBD581E080932901809100018823B8
:1008B00009F03CC082EF62E345D5182F8230B1F5D4
:1008C00082E3EBD58A3F91F5CE01029662E38BD5A8
:1008D000823021F5CE01039662E385D59A8182307C
:1008E000B1F49B3A31F48B81853819F040920001C4
:1008F00003C083E080930001792E66248B8190E011
:100900008629972990932101809320010FC040925E
:100910000001909320011092210108C01093000162
:1009200005C02092290181E080930001809100019F
:10093000882311F4409200016091200170912101FF
:10094000809100010E94BE150E94411780912901EB
:10095000823011F4F0D1F5D180910001833011F48F
:1009600088EFEED580E0B1DE8FB7F894A090360125
:10097000B0903701C0903801D09039018FBF8AE024
:100980000E9496118AE00E94961180EE92E00E94E9
:10099000B21180912001909121010E94AA118AE058
:1009A0000E94961185ED92E00E94B21180910001A3
:1009B000823061F0833018F4813089F405C08330CF
:1009C00049F0843061F408C081E301C082E30E94F1
:1009D000961109C083E3FBCF88EC92E002C080EC63
:1009E00092E00E94B21180912901823019F481EBCA
:1009F00092E002C081EA92E00E94B21188248394BE
:100A0000CE01019660E0EFD4882009F4DDC0823089
:100A100008F485C0823009F06DC019818091000111
:100A2000813069F41F3F09F44EC017FF05C0812FC4
:100A30008F7760E070DE64C0812F60E013C090911A
:100A40002401992309F1E92FF0E0EF5FFE4F808147
:100A5000181799F4E92FEF5FE0932401E33021F4B4
:100A60008EE761E05BDE4CC0E83009F049C08EE7FC
:100A700061E051DE1092240143C0933018F08EE7FC
:100A800061E049DE10922401103E91F0113E28F4FD
:100A90001123C9F01A3AE1F433C0103F29F01C3F8A
:100AA00079F0113EA9F408C081E08093220128C0AA
:100AB00081E08093230124C081E08093240120C041
:100AC00080E197E203C0F6DD88E893E160D518C0C5
:100AD00080912201882339F0812F609123011BDE50
:100AE0001092220104C0812F6091230117DE109221
:100AF000230106C08EEF62E325D49924939401C0AC
:100B000099248FB7F894A0903601B0903701C09027
:100B10003801D09039018FBF5524539471C0882378
:100B200009F06EC0992009F06BC00E943B1A182F83
:100B30000E943E1A082F079500270795012B8091E8
:100B40002501081709F45CC0FF24F394F022E02E7D
:100B5000E69421E0E222102F1695169511708091EF
:100B60002001909121016F2D70E02E2D30E0805BEF
:100B70009F4B41F4660F771F660F771F612B220F83
:100B8000331F07C0660F771F612B220F331F220F01
:100B9000331F622B8DEE9BD4FF0CFE28110F110F1B
:100BA000812F8F2992DD009325012AC08FB7F894F9
:100BB000A0903601B0903701C0903801D090390133
:100BC0008FBF5524539402C05520B9F02FB7F89425
:100BD0008091360190913701A0913801B09139018F
:100BE0002FBF8A199B09AC09BD09C397A105B1059F
:100BF00020F08AE00E94961155240E94F91702CE37
:100C000090DD882399F6E0CF1F920F920FB60F92D6
:100C100011248F939F9393B19F718091280198170E
:100C200029F0909328018AE08093090180910901BD
:100C3000882349F0815080930901882321F4809111
:100C40002801809327019F918F910F900FBE0F90E5
:100C50001F90189584B1807E84B985B18F6185B964
:100C6000E1E7F0E08081826080838AEF90E09093FA
:100C700099008093980010929000E1E9F0E088E0FC
:100C80008083808183608083089580912701089507
:100C90009C0180918100887F8093810080916F000A
:100CA0008D7F80936F00109285001092840082E007
:100CB00086BB2115310581F0220F331F3093890047
:100CC0002093880080916F00826080936F008091F4
:100CD00081008260809381000895882319F027980D
:100CE0002F9A08952F98279A0895882319F05098DD
:100CF000589A08955898509A0895382F4DB3E99806
:100D00000000882319F05198599A02C0519A5998B5
:100D100024E189B190E0969587958170831711F051
:100D20002150B9F782E08CBB41FF02C0E99A01C0B3
:100D3000E9988DB30895F894E99882E08CBB789493
:100D40000895F894E9E6F0E080818C608083E99A68
:100D500078940895882321F08091110180931201E5
:100D600089B190E096958795982F917080911201A6
:100D70008F3F21F481E08927809312018091120135
:100D8000813089F0813018F08E3FB9F419C0992371
:100D9000C9F08AE590E07CDF8EEF8093110181E05D
:100DA000809312010AC0992369F488EE93E070DF02
:100DB0008FEF809311011092120191E0892F089515
:100DC00092E001C094E08FEF80931201F7CF1F9360
:100DD00019B11170882321F080910A0180930B01D1
:100DE00080910B018230F1F0833020F4813009F0E2
:100DF0004BC006C0833079F18E3F09F045C03AC040
:100E00008EEF80930A0180EB94E042DF10922D0177
:100E100010922C01112311F416E02DC082E0809372
:100E20000B0132C017951127179580912C018695DB
:100E3000182B10932C0180912D018F5F80932D0131
:100E4000883011F513E010930A0188E790E020DF65
:100E500010930B0119C080E090E01ADF80912C0103
:100E600080932A0112E007C088EB9BE090D3109397
:100E70002B010AC015E080E090E00ADF81E080935A
:100E80000B01123089F7F3CF1F9108950F931F9331
:100E9000982F80910E018F3F19F482E080930E010C
:100EA000992321F080910D0180930E0180910E0114
:100EB000873009F460C0883088F4843009F43EC07B
:100EC000853030F48230E9F0833009F081C02CC0E5
:100ED0008530B1F1863009F07BC04BC08A3009F40F
:100EE0005FC08B3038F4883009F44FC0893009F086
:100EF0006FC04DC08B3009F457C08E3F09F068C0F9
:100F00005AC080912E0180932F0188E08093300198
:100F100081E080930C0183E080930D0188EC90E0E8
:100F2000B7DE80E0EADE54C080E0DFDE81E0E5DEAF
:100F30008EEF80930D0180E29EE4AADE85E031C051
:100F400010912F01012F0170802FCFDE1695109385
:100F50002F0180910C01802780930C01809130013A
:100F6000815080933001882311F084E01AC086E01C
:100F700018C087E016C080910C01B7DE8091300167
:100F800081508093300188E00CC089E00AC081E084
:100F9000ACDE809130018150809330018AE001C045
:100FA0008BE080930E0114C080E090E071DE4899E0
:100FB0002CC012E007C0109130011295107F15600F
:100FC000123030F081E091DE8FEF80930E0119C076
:100FD00089B120910E0130E02170307090E096953B
:100FE0008795817090702817390711F411E009C0B6
:100FF00081E07BDE8FEF80930E0188EB9BE0C7D210
:1010000014E0812F1F910F91089519E0DBCFFF921B
:101010000F931F93F9B099B1882329F08FEF809334
:10102000100115E07DC0809110018F3F19F481E01F
:1010300080931001092F0170109110011630E9F111
:10104000173040F41430D9F01530D8F4113009F0CD
:1010500050C008C01830D9F1183088F1193009F0A3
:1010600048C037C080EB94E013DE1092320110923A
:10107000310110930F01002309F057C01CC085E017
:1010800017C0902F97959927979580913101869554
:10109000982B9093310180910F01802780930F014D
:1010A000809132018F5F80933201883021F486E095
:1010B000809310011EC084E0FBCF87E0F9CF8091C0
:1010C0000F01801711F017E031C088E0F1CF89E0FF
:1010D000EFCF002349F08091310180932A0181E014
:1010E0008093290112E022C088EB9BE050D218E0E7
:1010F0001DC02091100130E0217030708F2D90E0E4
:1011000096958795817090702817390711F411E032
:1011100007C08FEF8093100188EB9BE038D214E07A
:10112000812F1F910F91FF90089516E080E090E0CD
:10113000AFDD8FEF80931001F3CFDF92EF92FF923C
:101140000F931F93082F8230F9F480912901823088
:1011500021F483E0809333016BC0809135018130AD
:1011600079F483E08093350180913301882319F06D
:1011700088EB9BE00CD281E08093330100E004C057
:1011800081E08093340154C0FF24F394A2E0DA2E6E
:10119000F3E0EF2E80913501813031F1813030F074
:1011A000823081F1833009F043C039C0802FD2DD15
:1011B000823008F43DC0823069F780913401882381
:1011C00079F01092340180913301882319F088EB73
:1011D0009BE0DDD1F0923301E092350100E0DACFFF
:1011E00081E08093350124C049991FC0809133016B
:1011F000882319F088EB9BE0CAD1F0922B01D092A2
:101200003501C8CF802F03DF182F823088F082305D
:1012100019F088EB9BE0BBD110932B0106C0802F07
:1012200035DE823028F08093330110923501B2CF41
:101230001F910F91FF90EF90DF9008951F920F92F2
:101240000FB60F920BB60F9211242F933F934F932B
:101250005F936F937F938F939F93AF93BF93EF931E
:10126000FF9380912901823019F480E0B0DD02C043
:1012700080E063DFFF91EF91BF91AF919F918F91DC
:101280007F916F915F914F913F912F910F900BBE86
:101290000F900FBE0F901F901895F89481E02DDDF0
:1012A00081E023DD1092800088E080938100E9E6F0
:1012B000F0E08081837F84608083E99A80E03DDF75
:1012C000789408951F920F920FB60F920BB60F925B
:1012D00011242F933F934F935F936F937F938F933B
:1012E0009F93AF93BF93EF93FF9380918100887F8B
:1012F0008093810080916F008D7F80936F0000004C
:10130000109285001092840082E086BB80912901B2
:10131000823019F481E05BDD02C081E00EDFFF91D5
:10132000EF91BF91AF919F918F917F916F915F915D
:101330004F913F912F910F900BBE0F900FBE0F90CA
:101340001F901895DF92EF92FF920F931F93182F23
:10135000D62E80912901823011F480E03EC087E7CB
:10136000E5D7812FEDD780E2E1D7F89410932E01D5
:101370001092330182E0E1DE78948FB7F894E09028
:101380003601F090370100913801109139018FBF7B
:101390004D2D50E060E070E018C0DD20B1F02FB7B7
:1013A000F8948091360190913701A0913801B09165
:1013B00039012FBF8E199F09A00BB10B4817590790
:1013C0006A077B0710F48AE008C0809133018230FD
:1013D00020F380913301109233011F910F91FF9000
:1013E000EF90DF900895DF92EF92FF920F931F939B
:1013F000CF93DF93EC018FB7F894E0903601F09033
:10140000370100913801109139018FBFD0902B0125
:101410006623C1F41FC02FB7F894809136019091D4
:101420003701A0913801B09139012FBF8E199F0962
:10143000A00BB10B481759076A077B0728F1D0901A
:101440002B0104C0462F50E060E070E081E08D1574
:1014500010F703C081E08D15B8F410912A011092A5
:101460002B0182E0D81651F482E760D7812F68D72C
:1014700080E25CD7209741F0188306C082E556D7FA
:101480008D2D5ED780E252D78D2DDF91CF911F91A8
:101490000F91FF90EF90DF9008951F93DF93CF930C
:1014A0000F92CDB7DEB7682FCE0101969CDF182FC3
:1014B000823039F0198282E539D781E337D7812F1D
:1014C0003FD789810F90CF91DF911F910895EF92BF
:1014D000FF920F931F93E82EF62E80912901823000
:1014E00049F103E08E2D62E32DDF182F8230D1F415
:1014F00082E3D3DF182F8A3F69F48F2D62E322DF66
:10150000182F823059F482E3C8DF182F8A3F11F474
:1015100081E011C081E20AD781E207C087E506D7E2
:1015200082E303C087E502D781E300D7812F08D784
:101530000150C1F680E01F910F91FF90EF90089548
:10154000FF920F931F93F82E809129018230D1F0E2
:1015500003E08F2D62E3F6DE182F823059F482E328
:101560009CDF182F8A3F11F481E00DC081E2DED6A6
:1015700081E203C087E5DAD680E3D8D6812FE0D6B2
:10158000015039F780E01F910F91FF9008959093DB
:101590003B0180933A015E9A0895EEE6F0E0808187
:1015A000826080838AEF87BD82E084BD15BC85B5EB
:1015B000836085BD08951F920F920FB60F920BB6F0
:1015C0000F9211242F933F934F935F936F937F93C9
:1015D0008F939F93AF93BF93EF93FF9380913601C7
:1015E00090913701A0913801B09139010196A11D68
:1015F000B11D8093360190933701A0933801B093C9
:10160000390180913A0190913B01009731F00197A7
:1016100090933B0180933A0101C05E9880913C0118
:10162000882341F481E080933C0178940E94DB1A86
:1016300010923C01FF91EF91BF91AF919F918F91DB
:101640007F916F915F914F913F912F910F900BBEC2
:101650000F900FBE0F901F9018952091150130919B
:1016600016012115310521F42DB73EB72052304027
:101670008091170190911801281B390BC901089519
:10168000AC0120911501309116012115310521F48D
:101690002DB73EB72052304080911701909118012C
:1016A000281B390B2417350718F420E030E007C059
:1016B000480F591F50931801409317019C01C9010D
:1016C00008958BEA93E09093180180931701089591
:1016D0001092490110924A0110924B0110924C0154
:1016E00010924D0110924E01E2E5F1E0119281E07D
:1016F000ED36F807D9F7109240018FE00895E8DF42
:1017000081E88093D70080EA8093D80086E189BD84
:1017100009B400FEFDCF80E98093D8001092E0006C
:101720001092420110923D0110923E0110923F0131
:101730008DE28093E2007894089580913F018823A0
:1017400061F080913E01882341F48091E000826045
:101750008093E00081E080933E010895582F382F58
:101760003150343A10F040E014C0E32FE695E6958E
:10177000E695F0E0EE5AFE4F232F277081E090E0CF
:1017800002C0880F991F2A95E2F72081282B208319
:1017900043E0852F885A8330A0F4E52FE695E6953F
:1017A000E695F0E0EE5AFE4F252F277081E090E09D
:1017B00002C0880F991F2A95E2F72081282B2083E9
:1017C0004460852F885E8831A8F4252F2853E22FA6
:1017D000E695E695E695F0E0EE5AFE4F277081E03B
:1017E00090E002C0880F991F2A95E2F72081282BEC
:1017F00020834860252F205E283080F481E090E02F
:1018000002C0880F991F2A95E2F7982F882331F09C
:1018100080914001892B8093400115C0343AD0F467
:10182000E9E4F1E080818517A9F0319681E0EF3499
:10183000F807C1F720E030E0F901E75BFE4F808157
:10184000882319F45083436005C02F5F3F4F263033
:10185000310591F7842F0895482F282F2150243ADD
:1018600010F030E014C0E22FE695E695E695F0E042
:10187000EE5AFE4F277081E090E002C0880F991F5A
:101880002A95E2F7809520818223808333E0842F9C
:10189000885A8330A8F4E42FE695E695E695F0E0C3
:1018A000EE5AFE4F242F277081E090E002C0880F8F
:1018B000991F2A95E2F780952081822380833460E6
:1018C000842F885E8831B0F4242F2853E22FE695C8
:1018D000E695E695F0E0EE5AFE4F277081E090E045
:1018E00002C0880F991F2A95E2F7809520818223F4
:1018F00080833860242F205E283050F481E090E00F
:1019000002C0880F991F2A95E2F7982F882319F4AF
:10191000E9E4F1E008C0909580914001892380932B
:10192000400133600AC08081841711F41082336053
:10193000319681E0EF34F807B1F7832F0895982F9F
:1019400080914201882309F492C090FF2EC02FB7E6
:10195000F89481E08093E9008091E80085FF24C03D
:10196000809140018093F1001092F1008091490133
:101970008093F10080914A018093F10080914B01A6
:101980008093F10080914C018093F10080914D0192
:101990008093F10080914E018093F1008AE380935F
:1019A000E800109248019E7F2FBF80911901882383
:1019B00009F45CC091FF20C02FB7F89482E08093B7
:1019C000E9008091E80085FF16C081E08093F10076
:1019D000809140018093F100E2E5F1E081918093F4
:1019E000F10081E0E736F807C9F78AE38093E80061
:1019F000109245019D7F2FBF92FF16C03FB7F8940C
:101A000022E02093E9008091E80085FF0CC020933C
:101A1000F100809167018093F1008AE38093E800F0
:101A2000109246019B7F3FBF93FF21C02FB7F894D0
:101A300082E08093E9008091E80085FF15C083E093
:101A40008093F100809168018093F1008091690199
:101A50008093F10080916A018093F1008AE3809382
:101A6000E80010924701977F2FBF01C0917F892F17
:101A70000895482F80914201882309F44DC0809138
:101A80003D01882309F048C080913E01882309F078
:101A900043C080911901882309F43EC02FB7F89400
:101AA00083E08093E90080915101882341F0809187
:101AB000E80085FD02C02FBF12C010925101909125
:101AC000E4009C5F33E08091E80085FD13C02FBFE8
:101AD0008091E400891729F481E0809351018FEF10
:101AE0000895809142018823B9F02FB7F89430937C
:101AF000E900E9CF4093F1008091E80085FD06C040
:101B00008AE38093E80010924F0103C082E0809343
:101B10004F012FBF80E008958FEF08951F920F921D
:101B20000FB60F920BB60F9211242F938F939F93A2
:101B3000EF93FF938091E1001092E100282F83FF43
:101B400017C01092E90081E08093EB001092EC0046
:101B500092E29093ED0098E09093F0001092420191
:101B600010923F0110923D0110923E0180931901A5
:101B700020FF08C08091E20080618093E20081E054
:101B800080933D0124FF0BC080913D01882339F0F3
:101B90008091E2008F7E8093E20010923D0125FF4C
:101BA00002C010923E0122FFDBC0809142018823D7
:101BB00009F4D6C0809119018823B1F080914F01BA
:101BC000882391F0815080934F01882369F483E04A
:101BD0008093E90002C01092F1008091E80085FD39
:101BE000FACF8AE38093E80080911901882371F08D
:101BF00080914401882319F08150809344018091A1
:101C00004301882319F08150809343018091500152
:101C10008F5F8093500190E083709070892B09F062
:101C20009FC090911D01992389F181E08093E90083
:101C30008091E80085FF2AC0809148018F5F8093E2
:101C40004801891718F11092480180914001809352
:101C5000F1001092F100809149018093F100809190
:101C60004A018093F10080914B018093F1008091B3
:101C70004C018093F10080914D018093F10080919F
:101C80004E018093F1008AE38093E800809119016E
:101C9000882309F465C082E08093E90090911A01DD
:101CA000992301F18091E80085FF1CC080914501D6
:101CB0008F5F809345018917A8F01092450181E05C
:101CC0008093F100809140018093F100E2E5F1E022
:101CD00081918093F10081E0E736F807C9F78AE344
:101CE0008093E80090911B019923B9F08091E8005E
:101CF00085FF13C0809146018F5F8093460189174D
:101D000060F01092460182E08093F10080916701BB
:101D10008093F1008AE38093E80090911C0199235D
:101D2000F9F08091E80085FF1BC0809147018F5F2B
:101D3000809347018917A0F01092470183E08093B8
:101D4000F100809168018093F10080916901809396
:101D5000F10080916A018093F1008AE38093E800AA
:101D6000FF91EF919F918F912F910F900BBE0F904C
:101D70000FBE0F901F9018951F920F920FB60F92E3
:101D80000BB60F9211242F933F934F935F936F9352
:101D90007F938F939F93AF93BF93CF93DF93EF93F3
:101DA000FF931092E9008091E80083FF4BC260919D
:101DB000F1003091F1008091F100482F50E0209126
:101DC000F100922F80E0482B592B8091F100A82F31
:101DD000B0E02091F100922F80E0A82BB92B8091E8
:101DE000F100C82FD0E02091F100922F80E0C82BA5
:101DF000D92B82EF8093E800363009F056C025EFEA
:101E000032E0B90165507040F9013797859194919E
:101E100084179507E1F4FB01859194918A179B073C
:101E2000B1F49B012E5F3F4FF901659174912E5FD4
:101E30003F4FF9012491CE01CF3FD10519F010F0A9
:101E40008FEF90E0422F821758F4482F09C0295F86
:101E50003F4F695F7F4FF3E020353F07A9F6F2C19E
:101E60005EEF8091E800282F30E0C9018570907006
:101E7000892BB9F322FDE9C1342F413208F030E259
:101E8000232FCB0106C0FC010196E491E093F10001
:101E900021502223C1F7630F711D431B5093E800AB
:101EA0004423F9F63032E9F2D0C1862F8F7709F05A
:101EB0005BC0353061F48EEF8093E8008091E800DC
:101EC00080FFFCCF842F80688093E300BEC139304F
:101ED00019F5409342018EEF8093E80089E493E086
:101EE00021E02093E900FC010196E491E093EB00EE
:101EF000EE2369F0AC014F5F5F4FFC01849180934A
:101F0000EC00CA010196FA0134913093ED002F5F85
:101F1000263039F78EE164C0383039F48091E8001A
:101F200080FFFCCF809142010AC1332341F48091AC
:101F3000E80080FFFCCF80913F01880F2BC031303B
:101F400019F0333009F07EC14130510509F07AC1F2
:101F50008EEF8093E800313019F410923F0175C183
:101F600081E080933F0171C1823009F03EC033238C
:101F7000B1F48091E80080FFFCCFA093E90080914C
:101F8000EB0090E025E0969587952A95E1F7817022
:101F90001092E9008093F1001092F1004FC13130AE
:101FA00019F0333009F04EC1452B09F04BC12A2FEF
:101FB0002F77822F8150853008F044C18EEF8093B7
:101FC000E8002093E900333009F43CC189E18093B3
:101FD000EB0081E090E002C0880F991F2A95E2F79C
:101FE0008093EA001092EA0030C1813209F02AC1E0
:101FF000A230B10509F06CC0E42F313069F5809151
:10200000E80080FFFCCFE13081F4E093F1008091A3
:1020100040018093F100E2E5F1E081918093F100CD
:1020200081E0E736F807C9F709C1E23029F4E09307
:10203000F1008091670183C0E33009F0FFC0E093B5
:10204000F100809168018093F10080916901809393
:10205000F10080916A0173C0393039F48091E80051
:1020600082FFFCCF8091F10073C0323071F4809117
:10207000E80080FFFCCFEE2329F0F0E0E75EFE4FA2
:1020800080815DC080911A015AC03A3009F0DAC0EF
:10209000442371F0A42FB0E01197FD01E65EFE4FDE
:1020A0005083552309F0CAC0AB5BBE4F1C92C6C01B
:1020B00050931A0150931B0150931C01552309F0B2
:1020C000BDC0109245011092460110924701B6C062
:1020D000109709F055C0313009F58091E80080FF74
:1020E000FCCF809140018093F1001092F10080912B
:1020F00049018093F10080914A018093F100809121
:102100004B018093F10080914C018093F10080910C
:102110004D018093F10080914E0111C0323039F4AD
:102120008091E80080FFFCCF80911D0108C0333012
:1021300049F48091E80080FFFCCF809119018093E1
:10214000F1007CC0393061F48091E80082FFFCCF5F
:102150008091F100809341018BEF8093E8006EC085
:102160003A3041F450931D01552309F067C0109295
:10217000480164C03B3009F065C0409319015EC05E
:10218000A130B10519F5313009F05CC04C2F5EEF7C
:102190008091E800282F30E0C90185709070892B6C
:1021A000B9F322FD52C0942F413208F090E2892FFA
:1021B00003C01092F10081508823D9F7491B509336
:1021C000E800442329F7903219F33FC01397D1F563
:1021D000313001F540E45EEF8091E800282F30E0D7
:1021E000C90185709070892BB9F322FD2EC0942F00
:1021F000413208F090E2892F03C01092F100815023
:102200008823D9F7491B5093E800442329F79032DB
:1022100019F31BC03930B1F490E42BEF8091E80042
:1022200082FFFCCF2093E800892F913208F080E2F2
:10223000981BA1F78091E80080FFFCCF8EEF809380
:10224000E80003C081E28093EB00FF91EF91DF9102
:10225000CF91BF91AF919F918F917F916F915F913E
:102260004F913F912F910F900BBE0F900FBE0F908B
:102270001F901895FC0180914201882339F12FB7F6
:10228000F8946093440185E08093E90095E08091A3
:10229000E80085FF02C090E40EC02FBF809144018A
:1022A0008823A9F080914201882381F02FB7F89408
:1022B0009093E900ECCF8091F10081939150D9F790
:1022C0008BE68093E8002FBF80E408958FEF089598
:1022D000FC0180914201882339F12FB7F894609373
:1022E000430184E08093E90094E08091E80085FF59
:1022F00002C090E40EC02FBF809143018823A9F053
:1023000080914201882381F02FB7F8949093E900DF
:10231000ECCF81918093F1009150D9F78AE38093BB
:10232000E8002FBF80E408958FEF0895A2CB0895B1
:10233000982F8A3010F087E301C080E3890F99CB92
:102340001F93182F82958F70F3DF812F8F70F0DF2E
:102350001F9108951F93182F892FF2DF812FF0DF2F
:102360001F9108951F93CF93DF93EC01FE012196F7
:102370001491112339F01A3011F48DE07ADB812F9A
:1023800078DBF4CFDF91CF911F910895382F209102
:102390007001E0916D01F0916E0190E009C0DF01E4
:1023A00080813296831719F411968C9108959F5F5E
:1023B0009217A8F380E008950F931F93CF93DF93B4
:1023C000182F062F809173018823B1F1662349F0FD
:1023D000E0917501F0917601E10FF11D809174019A
:1023E0008083C12FD0E0E0917501F0917601EC0F70
:1023F000FD1F8081CBDF282F8823F1F080917301AE
:102400008217D0F081E090E0821B9109880F991F1C
:10241000E0917101F0917201E81BF90B0190F081DC
:10242000E02DEC0FFD1F8081882311F0E82F09C0FB
:10243000C656DE4FE88105C0E12FF0E0E656FE4FBC
:10244000E0812E2F30E0C901887F9070803D91059A
:10245000D9F44091740127703070002349F081E075
:1024600090E002C0880F991F2A95E2F7482B09C017
:1024700081E090E002C0880F991F2A95E2F78095CD
:10248000482340937401E0E08E2FDF91CF911F919C
:102490000F91089510926F011092700110927301C4
:1024A00010926E0110926D011092720110927101E2
:1024B00010927601109275010895ECDF80E0815052
:1024C000E82FF0E0E656FE4F80838823C1F7089599
:1024D000382F2091700180916F01281778F4822F96
:1024E00090E0880F991FE0916D01F0916E01E80F67
:1024F000F91F308361832F5F20937001089510923C
:1025000074018091750190917601892B59F080E0DA
:102510008150E0917501F0917601E80FF11D108274
:102520008823B1F70895AF92BF92CF92DF92EF92D6
:10253000FF920F93DF93CF9300D0CDB7DEB75C014E
:10254000E62E80917301841770F1442329F46AE91F
:10255000C62E61E0D62E0EC081E090E0841B91096A
:10256000880F991FE0917101F0917201E81BF90B3E
:10257000C080D18000E015C0C50101969A8389838F
:10258000C5010E94271CF82EE2E0F0E0AE0EBF1E4F
:1025900089819A810E94271CF601EF0DF11D80832D
:1025A0000F5F0E1548F30F900F90CF91DF910F91B1
:1025B000FF90EF90DF90CF90BF90AF900895EF9293
:1025C000FF920F931F93CF93DF93E82EF62E66238F
:1025D00009F44FC080E091E053D890937601809346
:1025E00075018DDFCF2DD0E00E2D10E0CE01969538
:1025F000982F8827979587958C0F9D1F800F911F87
:10260000880F991F3DD89C0190936E0180936D01B6
:10261000009711F480E02EC0E0926F01F0927301F8
:10262000C801880F991F820F931F909372018093A6
:1026300071019E01220F331F280F391F90E040E0E7
:1026400050E015C0E0917101F0917201E40FF51FA7
:102650003183208380E08150F901E80FF11D108261
:102660008823C9F720503F4F9F5F4E5F5F4F9F15F4
:1026700048F381E0DF91CF911F910F91FF90EF9090
:10268000089581E080937C01089510927C01089563
:10269000582F40917B01E0917801F091790130E071
:1026A00014C08081851779F481812281922F9095C1
:1026B0009823962392959F70692B8627822319F47D
:1026C0002381348106C03F5F3596341750F320E0F4
:1026D00030E0C901089510927C0110927A011092A5
:1026E0007B018091780190917901892B21F01092E2
:1026F0007901109278010895EECF08951092770134
:1027000080919A0290919B02892B59F080E0815030
:10271000E0919A02F0919B02E80FF11D108288234C
:10272000B1F708957F928F929F92AF92BF92CF920E
:10273000DF92EF92FF920F931F93CF93DF93862E3A
:1027400090907A01C0917801D0917901AA2425E076
:10275000722E3DC0B0907B01B914D9F1B79C7001C5
:102760001124EC0EFD1E8C010F5F1F4F0E94271CD1
:10277000F701808368010894C11CD11CC8010E9424
:10278000271CF701818386010F5F1F4FC6010E943E
:10279000271CF70182831483038378010894E11CCA
:1027A000F11CC8010E94271C182FC7010E94271C7A
:1027B0008F731F73810F880F0894E11CF11C970120
:1027C000280F311DC901B394B0927B01A394A814C2
:1027D00008F2DF91CF911F910F91FF90EF90DF9062
:1027E000CF90BF90AF909F908F907F9008951F9350
:1027F000182F662349F080E091E00E94400B9093EF
:102800009B0280939A027ADF85E0189FC001112411
:102810000E94400B9093790180937801009711F406
:1028200080E005C010937A0110927B0181E01F9136
:102830000895BF92CF92DF92EF92FF920F931F9372
:10284000CF93DF93C62EB42E8C010F5F1F4FFFD79F
:10285000F82EE8012196C801FAD7D82E8F2D8F7354
:10286000BB2011F0E82E1BC04FE3E42EED2090E0DA
:10287000880F991FC80FD91FD7FE11C084E86C2D8F
:102880005AD60DC08E010F5F1F4FCE01E0D7F82E34
:102890002296C801DCD7682F8F2D4DD6EA94EE2002
:1028A00089F7BB2029F4D7FE03C088E060E043D657
:1028B000DF91CF911F910F91FF90EF90DF90CF901C
:1028C000BF900895FF920F931F93082FF62E10913B
:1028D0007701E0919A02F0919B02309761F06623B4
:1028E00019F0E80FF11D1083E0919A02F0919B021C
:1028F000E00FF11D108180917C01882351F0802F21
:10290000612FC6DE009729F0612F4F2D92DF51E035
:1029100001C050E0202F30E0C901887F9070803ED8
:102920009105D1F44091770127703070FF2049F074
:1029300081E090E002C0880F991F2A95E2F7482BAA
:1029400009C081E090E002C0880F991F2A95E2F744
:102950008095482340937701852F1F910F91FF9019
:10296000089580917D0190E0882309F491E0892FFA
:1029700008959C0151E050939F0280917D0188232E
:1029800011F08FEF0895F99B02C08EEF08957093B8
:102990009D0260939C023093A1022093A002409379
:1029A0009E0250937D01FB9A80E008951F920F9242
:1029B0000FB60F920BB60F9211242F933F934F93A4
:1029C0005F936F937F938F939F93AF93BF93EF9397
:1029D000FF9380919E02882329F180919F02882392
:1029E00091F180919C0290919D0231D724C08091F9
:1029F0009E02815080939E028091A0029091A1023C
:102A000001969093A1028093A00280919C029091E4
:102A10009D02019690939D0280939C0280919E025C
:102A2000882321F4FB9810927D0132C080919C0292
:102A300090919D020CD7982FE091A002F091A102F5
:102A400080819817A1F280919C0290919D0292BD85
:102A500081BDE091A002F091A102808180BDFA9A2F
:102A6000F99A80919E02815080939E028091A002EB
:102A70009091A10201969093A1028093A00280916F
:102A80009C0290919D02019690939D0280939C02DE
:102A9000FF91EF91BF91AF919F918F917F916F9136
:102AA0005F914F913F912F910F900BBE0F900FBEF2
:102AB0000F901F901895E2E0F0E089E080935700B6
:102AC000849183FD5AC0F89481E08093E00080E215
:102AD0008093D8001092C90080E29EE40197F1F73C
:102AE0001DBA109268001CBC10BE1FBA10927A006A
:102AF00010926E0010926F00109270001092710090
:102B00001092C9001092BC0011B814B817B81AB8C6
:102B10001DB810BA12B815B818B81BB81EB811BA3B
:102B2000E3E0F0E089E08093570084918670869519
:102B300093E0892720E034E002C0220F331F8A95FA
:102B4000E2F788E02030380791F088E0213038073C
:102B500020F42050344089F408C080E12030380748
:102B600041F02050304249F406C00C9400FE0C9411
:102B700000FC0C9400F80C9400F0089580938201FE
:102B800070938401609383010895282F285D69F074
:102B900081E090E002C0880F991F2A95E2F720910A
:102BA0001F01282720931F01089581E080931F01B2
:102BB00008951F9380E090E04AD6182F81E090E0BE
:102BC00046D620E093E4982783E58127982B09F4E3
:102BD00021E0822F1F910895ECDF882389F082E0A5
:102BE00090E03DD69C01009759F0275F3F4044F4A8
:102BF00084E090E02CD6813019F486E090E027C67E
:102C000080E00895EF92FF920F931F93CF93DF938D
:102C1000E62E142F00E020C0153010F1EC012496B0
:102C2000039615D6F82ECE0112D6982F9F7329F051
:102C3000809181018F5F809381012F2D2F73290F48
:102C4000220F412F4550421758F0CE010196820FB6
:102C5000911D142F121B0F5F0E15F0F281E001C0C1
:102C600080E0DF91CF911F910F91FF90EF90089539
:102C700083E090E060E0F8D582E090E060E0F4D599
:102C800081E090E063E4F0D580E090E063E5ECC59E
:102C900090DF882309F4ECCF0895AF92BF92DF92C2
:102CA000EF92FF920F931F93CF93DF93E62ED42ED4
:102CB000EC012196CE01CBD5082F182F1770DD20FF
:102CC00081F4113041F0113018F0123051F406C087
:102CD00081EF95E005C089EE95E002C081EE95E0B8
:102CE00041DB402F50E020911F0130E0CA01887382
:102CF0009070E3E095958795EA95E1F702C03595E8
:102D000027958A95E2F720FD06C0DD2009F0AEC0C8
:102D100088ED95E02FC021967EEFF72EFE0C06FF82
:102D200019C0CE0194D590E02091820130E021506D
:102D3000304002C0959587952A95E2F780FD06C040
:102D4000DD2009F093C082ED95E014C021966DEF6F
:102D5000F62EFE0C07FF13C0CE0181D52091830112
:102D6000309184018217930739F0DD2009F07EC08D
:102D70008DEC95E0F7DA7AC022962EEFF20E113044
:102D800009F43BC0113020F0123009F068C052C085
:102D9000CE015DD5482FA82EBB249501220F331FED
:102DA000FA948F2D90E02817390719F086EC95E0FA
:102DB00055C0DD2029F480917E01840F80937E012F
:102DC000219600E010E015C0CE0141D5F82ECE01CD
:102DD00001963DD5682FDD2019F08F2D79DB06C0D7
:102DE00080917F01861710F460937F0122960F5F18
:102DF0001F4F0A151B0544F339C08E010F5F1F4F8B
:102E0000CE0125D5E82EC80122D5682F90E0880F85
:102E1000991F2EEFF20E2F2D30E08217930719F035
:102E20008FEB95E01BC0DD2009F1C80101964E2D06
:102E30007ADB1CC08E010F5F1F4FCE0108D5E82E34
:102E4000DD2021F0C8016E2D6DDC10C0C8016E2D93
:102E50004F2DD8DE882329F488EB95E083DA80E0D3
:102E600006C0809180018E0D8093800181E0DF910A
:102E7000CF911F910F91FF90EF90DF90BF90AF9097
:102E80000895EF92FF920F931F93CF93DF9334DC5B
:102E900014DB0E94610B10927E0110927F01109250
:102EA00080011092810185DE882309F49AC082E0B6
:102EB00090E0D5D48C01FCEFEF2EFFEFFF2EE80E53
:102EC000F91E8AEA95E04EDAC70144DA8AE02EDA82
:102ED00005501040065F1F4008F083C084E090E07A
:102EE000B6D4813009F07DC085E090E0B0D4823066
:102EF00008F077C0C8E0D0E020C0CE01A8D4182FD9
:102F00001FDA80E413DACE0125DA80E20FDA153019
:102F100018F483EA95E042C0CE01612F40E0BDDEA7
:102F2000882319F48BE995E039C08AE0FFD9812F15
:102F300090E0C80FD91FE81AF90A1E141F04ECF21A
:102F40008FE895E00FDA80917E01FAD98AE0EED918
:102F500083E895E007DA80917F01F2D98AE0E6D92B
:102F600084E795E0FFD980918001EAD98AE0DED933
:102F700080917E0160917F0122DB882319F485E630
:102F800095E00CC0809180016091810130DC882344
:102F900039F480DA0E94610B86E595E0E3D921C01F
:102FA0008BE495E0DFD982E090E059D48C010450A5
:102FB0001040C8E0D0E00FC0CE0149D4F82ECE01B9
:102FC0006F2D41E06ADE882361F08F2D90E0C80FFD
:102FD000D91F081B190B1016110674F352DB81E080
:102FE00001C080E0DF91CF911F910F91FF90EF9092
:102FF0000895CF92DF92EF92FF920F931F93CF939A
:10300000DF93C090890123E0C21609F413C12C1587
:1030100040F081E0C81609F4DAC08C1508F4DDC070
:103020000CC0E5E0CE1609F451C1CE1608F440C13B
:10303000F6E0CF1609F0ACC189C183EA92E060E006
:1030400019D918160CF0B6C01091A302123009F469
:103050003BC0133020F4113009F0ACC007C013306E
:1030600009F463C0143009F0A5C089C0E9EFF5E0A8
:10307000A3EAB2E084918D93319626E0E231F20723
:10308000C9F782E090E0EBD3EC01009759F084E0BF
:1030900090E0DDD3182F85E090E0D9D31093AD02F6
:1030A0008093AE02882799278C1B9D0B8450904FEC
:1030B0008093B9029093BA020E942D0B8093B302C1
:1030C0009093B40282E02AC03091A50220E0809162
:1030D000A40290E0822B932B90938B0180938A0122
:1030E000875F9F40D0F484E090E090938D018093BF
:1030F0008C0110928F0110928E018EE891E062E0B7
:1031000070E042E036DC882341F41093A20282EAA8
:1031100092E060E0DDD8B9DA5EC081E08093A2027F
:1031200082EA92E060E0D4D845C082E090E09093DB
:103130008D0180938C018AE891E062E070E042E0CA
:1031400050E075D320918A0130918B01FFE0273F39
:103150003F0718F780918C0190918D010296909312
:103160008D0180938C012093A3023093A40282E00E
:103170008093A20282EA92E060E0AAD8E5C08FB70D
:10318000F8942091360130913701409138015091E7
:1031900039018FBF209390013093910140939201A8
:1031A0005093930182E08093A20282EA92E060E071
:1031B0008FD8E8C090911F0180911E01981709F4E3
:1031C000E4C05FDE80911F0180931E01DEC0C9DB79
:1031D000882309F04EC081E0D9C083EA92E060E024
:1031E00049D818160CF04CC08091A302823809F01F
:1031F00057C01091A402212F30E080918A01909154
:103200008B018217930708F44BC060918C01709179
:103210008D0187EA92E0412FACDB882309F040C0A2
:103220001093940182E08093A20282EA92E060E02F
:103230004FD803C096DB882311F483E0A7C0C09168
:103240008C01D0918D01D0909401A7EAEA2EA2E0E2
:10325000FA2E8E0109C0C801FAD2F70191917F01BF
:103260008917F1F40F5F1F4F802F8C1B8D1598F37A
:10327000BDC083E08093A20282EA92E060E028D899
:1032800082E084C02450304030938F0120938E011F
:103290008EE891E062E070E042E06BDB882359F059
:1032A00081E08093A20282EA92E060E011D86DC0D2
:1032B00058DB882311F484E069C084E08093A20283
:1032C00082EA92E060E004D8DCDD5FC083EA92E04D
:1032D00060E00E943A111816BCF58091A302833079
:1032E00031F0843009F451C0813071F54EC0009145
:1032F0008A0110918B010115110531F1013411057D
:1033000008F000E410E060918C0170918D0183EA77
:1033100092E0A8018CD283EA92E060E00E946811FA
:1033200080918A0190918B01801B910B90938B016E
:1033300080938A0180918C0190918D01800F911F63
:1033400090938D0180938C0185E020C08FB7F89415
:103350002091360130913701409138015091390167
:103360008FBF8091900190919101A0919201B091B5
:103370009301281B390B4A0B5B0B295E33404040FD
:10338000504010F486E002C096DB80E08093890113
:103390008FB7F89420913601309137014091380170
:1033A000509139018FBF80918901882311F08C15CC
:1033B00049F0209385013093860140938701509313
:1033C00088012AC08091850190918601A091870192
:1033D000B0918801281B390B4A0B5B0B29583341EC
:1033E00040405040C8F01092890116C02D2D30E0A9
:1033F00080918A0190918B01821B930B90938B019A
:1034000080938A012C0F3D1F30938D0120938C01F6
:10341000892B09F02ECF36CFDF91CF911F910F91DD
:10342000FF90EF90DF90CF900895982F977021E054
:1034300030E001C0220F9A95EAF786958695869529
:1034400090E0662351F0FC01ED51FD4F9081822FF9
:10345000892379F4292B20830895FC01ED51FD4F38
:103460009081822F892329F020952923208380E0D1
:10347000089581E008958091410108958091190196
:1034800008950E947F0B04DC18C8E3EEF2E011926D
:1034900083E0E330F807D9F732D830D987C08BE022
:1034A00060E049C01F93182F60E0BFDF8823B9F4A4
:1034B0008DE20E949611812F0E94A01180E20E944D
:1034C0009611812F60E00E94DC11182F882339F0BB
:1034D00060E0F8D9882319F483E0612F2CD01F9184
:1034E00008951F93182F61E0A0DF8823B9F48BE2C1
:1034F0000E949611812F0E94A01180E20E949611D5
:10350000812F61E00E94DC11182F882339F061E0DF
:10351000D9D9882319F482E0612F0DD01F91089525
:103520008091960190E0019720919501821B91096D
:1035300060E570E055C10F931F93082F162FF0DF41
:103540008823B1F08091950190E0FC01EE0FFF1F00
:10355000E55FFC4F412F50E0302F20E0422B532BF2
:1035600051834083019660E570E03AD180939501E4
:103570001F910F910895909196018091950189175F
:1035800019F4E0E0F0E010C0892F90E0FC01EE0FAC
:10359000FF1FE55FFC4F0190F081E02D019660E593
:1035A00070E01ED180939601CF010895809195011E
:1035B0008093960108950F931F9380913D01882376
:1035C00021F480913E01882391F080913E0188236F
:1035D00009F003C19091950180919601981709F423
:1035E000FCC00E949D0B8AE080939801F6C08091F8
:1035F0009801882361F0815080939801882309F015
:10360000ECC043DF0E94680B80939901E6C0E09113
:103610009601809195018E1719F4E0E0F0E008C062
:10362000F0E0EE0FFF1FE55FFC4F0190F081E02D11
:103630008F01F7FF0FC090919701983050F4E92F58
:10364000F0E0ED5FFC4F8091400180839F5F90939D
:1036500097011F77113091F11A3009F48EC08BDF7A
:10366000163009F469C0173090F4133009F44AC0D9
:10367000143030F4113011F1123009F09AC02EC01C
:10368000143009F452C0153009F093C051C01930FC
:1036900009F467C01A3038F4173009F452C01830F2
:1036A00009F087C052C01B3039F01B3008F465C0E8
:1036B0001C3009F07EC077C010E077C0E091960121
:1036C000809195018E1751F0F0E0EE0FFF1FE55F3E
:1036D000FC4F802F90E0936091838083802F887FC0
:1036E000883D19F4802F51DA64C084E60E94961157
:1036F000802F0E94A01180E20E949611802F0E94CC
:10370000AE0B11C0802F887F883D09F452C085E739
:103710000E949611802F0E94A01180E20E949611B3
:10372000802F0E942C0C982F45C00093400123C08D
:1037300080914001802B1DC0009580914001802325
:1037400018C080914001802714C0E0919701EE23BA
:1037500081F1E150E0939701F0E0ED5FFC4F808153
:1037600008C080919701882321F1109297018091E0
:1037700003038093400193E01DC0902F915089F086
:10378000E0919601809195018E1799F0F0E0EE0F8F
:10379000FF1FE55FFC4F892F90E09A609183808343
:1037A00008C0E9DE06C071DE11E00E94680B982FA8
:1037B00002C090E010E080919901892B80939901DB
:1037C000882321F00E949F0C80939901112329F0F6
:1037D00080E29EE40197F1F76ED91F910F91089551
:1037E00097FB092E07260AD077FD04D00CD006D00F
:1037F00000201AF4709561957F4F0895F6F7909523
:1038000081959F4F0895AA1BBB1B51E107C0AA1FBA
:10381000BB1FA617B70710F0A61BB70B881F991F71
:103820005A95A9F780959095BC01CD010895DC01CA
:10383000CB01FC01F999FECF06C0F2BDE1BDF89ABB
:10384000319600B40D9241505040B8F70895F9995F
:10385000FECF92BD81BDF89A992780B50895A8E161
:10386000B0E042E050E0E5CF262FF999FECF1FBA35
:1038700092BD81BD20BD0FB6F894FA9AF99A0FBE99
:0838800001960895F894FFCFB2
:1038880004E11477E1F014F0770AFE0101FFFF016B
:10389800FFFFFFFF7F0000AB03017D7D7D7D010100
:00000001FF
